:100000000000000000000528090083120313850189
:100010008601870183160313850002308D309F000F
:100020000F3085000230860018308700B101B20120
:10003000BD01BE018312031381309F008B010714A1
:100040008714071506112823903098008316031390
:10005000181598161F309900831203130611D61035
:100060001E3033211821D614BE20E92007210615A1
:10007000003040380A21003080380A2100309C20AE
:10008000013040380A21003080380A210F309C208E
:10009000023040380A21003080380A211E309C206E
:1000A0000611033040380A21003080380A212D30F3
:1000B0009C20043040380A21003080380A213C302E
:1000C0009C20053040380A21003080380A214B300E
:1000D0009C203D233428831203131F129F125619AC
:1000E0009F15561D9F1100001F1405231F15D613C1
:1000F0001F197828831203131E0883160313B100F7
:10010000B5001E08B200B60083120313D61E98284D
:10011000831603130230B3000030B400D222B11FA3
:10012000982883120313D61783160313B109B20953
:10013000831203131F10080083120313BA003A0836
:100140004121AF00BA0AFF39031908002F08242102
:100150009F280800B001FF240C21B00AFF240C21C5
:10016000B00AFF240C21B00AFF240C21B00AFF249E
:100170000C21B00AFF240C21B00A0800CB2050301B
:100180004B23D62050304B23DB2050304B23E9202B
:1001900050304B23080013308316031393000030B4
:1001A00094008312031328309400080007111323CE
:1001B00007150000080021300A2190300A2105307F
:1001C0000A2113300A2120300A2113230C300A217E
:1001D0000800003001210030FE2008300A210830DC
:1001E000AD003F30AE0000300C21AE0BF328AD0B5C
:1001F000F128003001210030FE20080080380A215B
:10020000080040380A2108000D300A2108000C308F
:100210000A21080087100000071093008C1D0E298A
:100220008C11000007140000000087140000080073
:10023000831203130D302C210A302C210800831265
:10024000031309302C21080083120313AF00D618C2
:10025000AA20D61C2C2108008312031364000C1E54
:100260002F299900080083120313BA003A0841218C
:10027000AF00BA0AFF39031908002F0824213629D4
:100280000800831203178D00831603178C130C14B8
:10029000831203170C088312031308006400750807
:1002A00003195C290C1C5C291010F50B582900342B
:1002B0000C100B308F0010148C1E4E291A080800E9
:1002C000831603133108AF003208B0002F0EF03848
:1002D000A500A507E23EA600323EA8002F080F3970
:1002E000A607A607A807E93EA700A707A707300E9D
:1002F0000F39A707A807A70DA80DA809A80D300852
:100300000F39A807A50D0730A4000A30A807A703D6
:10031000031C8629A707A603031C8A29A607A50391
:10032000031C8E29A507A403031C9229831203131F
:10033000D61EBE292B30D61B2D3024218316031345
:100340002508031DA8298312031320302421AC297A
:1003500083120313303E2421831603132608303EF4
:1003600024212E302421831603132708303E242114
:10037000831603132808303E24210800561EC52981
:10038000831603132408303E242183160313250803
:10039000303E2421831603132608303E2421831681
:1003A00003132708303E2421831603132808303E08
:1003B000242120302421080083120313240E0F3936
:1003C000031DE4292030E529303E242124080F397B
:1003D000303E24212F302421250E0F39303E242198
:1003E00025080F39303E24212030242120302421BB
:1003F000220E0F39031DFE292030FF29303E242113
:1004000022080F39303E242148302421210E0F3993
:10041000303E242121080F39303E24214D30242143
:10042000200E0F39303E242120080F39303E242180
:100430005330242108001C2A1D2A1E2A1F2A202A84
:10044000212A222A232A242A252A262A272A282A38
:10045000292A2A2A2B2A2C2A2D2A2E2A2F2A302AE8
:10046000312A322A332A342A352A08008316861381
:100470008312861706171B2286131B2206130800F9
:10048000831686138312861306171B22861708000D
:1004900083168613831286131B2206171B2206134C
:1004A000080083168613831286171B2206171B2249
:1004B000061308008316861783121B2206171B22B9
:1004C0000315861B0311061308007C221B228522BC
:1004D0001B22080086178316031300008617831259
:1004E00003131B22080083160313861383120313BE
:1004F000000086131B220800061783160313000052
:100500000617831203131B22080083160313061316
:100510008312031306131B220800CB010830CD0001
:100520006A227C22861F952A982A0310CB0D9C2ACA
:100530000310CB0DCB0A9C2A8522CD0B912A0800F3
:10054000CA000830CD000310CA0D031CA82AAC2A2B
:10055000732265226A22AF2A6A226522AF2ACD0B56
:10056000A32A08000310B901BA011030A100B20D8E
:10057000B10DBA0DB90D33083902031DC12A340873
:100580003A02031CC92A3408BA023308031CB30F09
:10059000B902BC0DBB0DA10BB72A3B08B1003C084A
:1005A000B20008008316031303103408B2023308A4
:1005B000031C330FB1020800FB220310C20CC10C54
:1005C000031CE82A3B08BD070318BE0A3C08BE0707
:1005D000BE0CBD0CC00CBF0CC30BDE2A042B441098
:1005E0003B08BD070318BE0A031844143C08BE07A5
:1005F0004418031408001030C3003E08C2003D0830
:10060000C100BE01BD01080008000130B600013084
:10061000B7001430B800442B0130B6000130B700E9
:100620005030B800442B0130B6000430B7003230EF
:10063000B800442B0130B6002030B700CC30B800F1
:10064000442B0130B6005030B7000130B800442BC5
:100650000230B6007730B7000130B800442B0430C8
:10066000B6003130B7000130B800442B1030B6006E
:100670000E30B7003830B800442B2030B600283098
:10068000B700DA30B800442BB80B442BB70B442B1F
:10069000B60B442B0800AC001323AC0B4C2B08000A
:0209FE002F08C0
:100A0000BB000030BC00BE000630BD00DC2205305B
:100A10008A001430B30040088A073F0830070318E3
:100A20008A0AB30703188A0A8207003400340034A4
:100A30000034003400340034003400340034003416
:100A40000034003400340034003400340034003406
:100A500000340034003400340034003400340034F6
:100A600000340034003400340034003400340034E6
:100A700000340034003400340034003400340034D6
:100A800000340034003400340034003400340034C6
:100A900000340034003400340034003400340034B6
:100AA00000340034003400340034003400340034A6
:100AB0000034003400340034003400340034003496
:100AC0000034003400340034003400340034003486
:100AD0000034003400340034003400340034003476
:100AE0000034003400340034003400340034003466
:100AF0000034003400340034003400340034003456
:100B00000034003400340034003400340034003445
:100B10000034003400340034003400340034003435
:100B20000034003400340034003400340034003425
:100B30000034003400340034003400340034003415
:100B40000034003400340034003400340034003405
:100B500000340034003400340034003400340034F5
:100B600000340034003400340034003400340034E5
:100B700000340034003400340034003400340034D5
:100B800000340034003400340034003400340034C5
:100B900000340034003400340034003400340034B5
:100BA00000340034003400340034003400340034A5
:100BB000003400340034003400345F340034003436
:100BC0000034003407340034073400340034143463
:100BD0007F3414347F341434003424342A347F3482
:100BE0002A3412340034263416340834343432347F
:100BF00000347634493455342234503400340034CF
:100C00000034053403340034003400341C342234FE
:100C10004134003400340034413422341C34003474
:100C20000034143408343E340834143400340834A6
:100C300008343E340834083400340034503430343E
:100C400000340034003408340834083408340834DC
:100C50000034003460346034003400340034203414
:100C6000103408340434023400343E3451344934EE
:100C700045343E340034003442347F344034003450
:100C80000034423461345134493446340034213420
:100C9000413445344B343134003418341434123474
:100CA0007F341034003427344534453445343934E6
:100CB00000343C344A34493449343034003401344B
:100CC000013479340534033400343634493449343A
:100CD00049343634003406344934493429341E3416
:100CE00000340034363436340034003400340034F8
:100CF00056343634003400340034003408341434AC
:100D0000223441340034143414341434143414347C
:100D100000344134223414340834003400340234B2
:100D2000013451340934063400343E3441344934FA
:100D300055345E3400347E341134113411347E3431
:100D400000347F34493449344934363400343E3435
:100D5000413441344134223400347F34413441340D
:100D600022341C3400347F3449344934493441340A
:100D700000347F34093409340934013400343E34FA
:100D80004134493449343A3400347F340834083427
:100D900008347F340034003441347F34413400342B
:100DA00000342034413441343F34003400347F3443
:100DB000083414342234413400347F344034403415
:100DC0004034403400347F3402340C3402347F34F5
:100DD00000347F340434083410347F3400343E341B
:100DE0004134413441343E3400347F3409340934D1
:100DF0000934063400343E344134513421345E34F5
:100E000000347F34093419342934463400344634EC
:100E100049344934493431340034013401347F34A5
:100E20000134013400343F344034403440343F34E2
:100E300000341F342034403420341F3400343F3415
:100E400040343C3440343F34003463341434083488
:100E500014346334003407340834703408340734ED
:100E6000003461345134493445344334003400345F
:100E70007F344134413400340034023404340834C3
:100E80001034203400340034413441347F34003491
:100E90000034043402340134023404340034403465
:100EA000403440344034403400340034013402349F
:100EB00004340034003420345434543454347834FA
:100EC00000347F34483444344434383400343834C3
:100ED00044344434443420340034383444344434C6
:100EE00048347F340034383454345434543418344F
:100EF000003408347E3409340134023400340834B8
:100F00005434543454343C3400347F34083404347E
:100F1000043478340034003444347D3440340034B4
:100F200000342034403444343D34003400347F34C1
:100F300010342834443400340034003441347F34D5
:100F40004034003400347C340434183404347834AD
:100F500000347C34083404340434783400343834B5
:100F6000443444344434383400347C341434143439
:100F700014340834003408341434143418347C34F1
:100F800000347C34083404340434083400344834E5
:100F90005434543454342034003404343F3444340E
:100FA0004034203400343C344034403420347C34E9
:100FB00000341C342034403420341C3400343C349D
:100FC0004034383440343C34003444342834103411
:100FD0002834443400340C345034503450343C34CD
:100FE00000344434643454344C34443400340034D5
:100FF00008343634413400340034003400347F3453
:1010000000340034003400344134363408340034C1
:101010000034083408342A341C34083400340834CA
:0A1020001C342A340834083400346C
:02400E00323D41
:104200003134363446343834373437342034623439
:104210006F346F3474346C34643472340034513419
:104220003D34313430344D3468347A3420343134D0
:104230003934323430343034623400344E346F34F4
:104240006B346934613420343334333431343034B2
:1042500020344C34433444340034363478343134EC
:10426000343463342034303438342F3430343434FC
:104270002F343134393400345034613475346C3473
:1042800066346A3475346A346F3466347234653433
:1042900065342034003431343234333434343534FA
:1042A00036343734383439343034313432343334CA
:1042B00034340034363465346D3420346C3469342D
:1042C00067346E3465342E342E342E342E342E342E
:0242D0000034B8
:00000001FF
